S0220000687474703A2F2F737265636F72642E736F75726365666F7267652E6E65742F1D
S12300000C9438000C9407190C94861F0C945F000C945F000C945F000C945F000C945F0004
S12300200C945F000C941B220C945F000C94B6250C945F000C94DB190C94B5190C9462184B
S12300400C94B6260C945F000C9435260C945F000C9455270C941D270C945F000C945F0029
S12300600C945F000C945F000C945F000C945F0011241FBECFEFD0E1DEBFCDBF14BEA895C7
S123008088E10FB6F89480936000109260000FBE15E0A0E0B1E0E4E2F2E502C005900D92C7
S12300A0A832B107D9F716E0A8E2B5E001C01D92A93FB107E1F70E94CA110C9411290C94E6
S12300C0000020E030E0D901AC54BF4F0E94F328802DF901ED5BFE4F80832F5F3F4F203AB2
S12300E0310589F720E030E0D901A857BE4F0E94F328802DF901E45CFE4F80832F5F3F4F40
S12301002530310589F712BC11BC089520E030E0F901ED5BFE4F8081D901AC54BF4F082EDA
S12301200E9400292F5F3F4F203A310589F712BC11BC0895199B11C020E030E0D901509637
S12301400E94F328802DF901ED51FE4F80832F5F3F4F203A310591F0F1CF20E030E0D901D2
S1230160A859BD4F0E94F328802DF901ED51FE4F80832F5F3F4F203A310589F712BC11BCB5
S12301800895199B11C020E030E0F901ED51FE4F8081D9015096082E0E9400292F5F3F4FC6
S12301A0203A310591F0F1CF20E030E0F901ED51FE4F8081D901A859BD4F082E0E940029EC
S12301C02F5F3F4F203A310589F712BC11BC089520E931E0D9010E94F328802D2055314073
S12301E0F901ED57FD4F80832F5A3E4F81E0203F380781F712BC11BC089520E430E0F9019B
S1230200ED57FD4F8081D901A05BBE4F082E0E9400292F5F3F4F203A310589F712BC11BC9F
S12302200895A2E0B0E00E94F328802D90E090931E0180931D0120911D0130911E01A3E08C
S1230240B0E00E94F328802D90E0982F8827820F931F90931E0180931D01ADEEB3E00E9434
S1230260F328802D90E090932201809321012091210130912201AEEEB3E00E94F328802D77
S123028090E0982F8827820F931F909322018093210180911D0190911E01909320018093F0
S12302A01F01A4E0B0E00E94F328802D90E090932401809323012091230130912401A5E06D
S12302C0B0E00E94F328802D90E0982F8827820F931F9093240180932301A6E0B0E00E94C0
S12302E0F328802D90E090930101809300012091000130910101A7E0B0E00E94F328802D93
S123030090E0982F8827820F931F9093010180930001A1E0B0E00E94F328802D80932805BC
S1230320A8E0B0E00E94F328802D80931301A9E5B1E00E94F328802D80932D01A2E0B4E030
S12303400E94F328902D892F8150843078F080912D01843039F481E08093180183E6809351
S1230360FA0506C082E08093180102C090931801A9E0B0E00E94F328802D80931201AEE0F1
S1230380B0E00E94F328802D80932601ABE0B0E00E94F328802D80931901A3E0B4E00E94BA
S12303A0F328802D80931A01ACE0B0E00E94F328802D80931B01AFE6B1E00E94F328802DFE
S12303C080931C01A2EFB1E00E94F328802D80939C0580919C05882319F081E080939C052E
S12303E0ADE0B0E00E94F328802D26E0829FC00111249093150180931401A1E7B1E00E9439
S1230400F328802D80931E06A0E7B1E00E94F328802D80931C068AE080934B0681E08093E0
S12304204906AFE8B1E00E94F328802D80932E0180912E0181FF05C080912E01827F8093BC
S12304402E0180912E0185FF05C080912E018F7280932E01A4EFB1E00E94F328802D90E05F
S12304602CE231E0AC01429FC001439F900D529F900D11249093F5058093F405A5EFB1E07A
S12304800E94F328802D8093F105A6EFB1E00E94F328802D8093EF05A7EFB1E00E94F3286A
S12304A0802D8093EE05A8EFB1E00E94F328802D90E09093ED058093EC052091EC05309107
S12304C0ED05A9EFB1E00E94F328802D90E0982F8827820F931F9093ED058093EC05ABEFB7
S12304E0B1E00E94F328802D90E09093300180932F0120912F0130913001ACEFB1E00E9455
S1230500F328802D90E0982F8827820F931F9093300180932F01ADEFB1E00E94F328802DB8
S123052090E090933201809331012091310130913201AEEFB1E00E94F328802D90E0982F06
S12305408827820F931F9093320180933101AFEFB1E00E94F328802D90E09093B604809311
S1230560B5042091B5043091B604A0E0B2E00E94F328802D90E0982F8827820F931F909311
S1230580B6048093B50420E030E0D901A25ABE4F0E94F328802DF901ED5DFC4F8083D90108
S12305A0AE58BE4F0E94F328802DF901E550FA4F8083D901A458BE4F0E94F328802D808BE7
S12305C02F5F3F4F2A30310501F7A7E0B2E00E94F328802D80933701A3E0B2E00E94F328D3
S12305E0802D8093380120E030E0F901E85DF94F84E6808BD901A45EBD4F0E94F328802DA0
S123060080832F5F3F4F2031310579F720E030E0D901A759BE4F0E94F328802DF901E85D20
S1230620FE4F80832F5F3F4F2430310589F720E030E0D901A25DBD4F0E94F328802DF901E7
S1230640E650FB4F80832F5F3F4F2031310589F7ADE6B1E00E94F328802D80932501A1EF99
S1230660B1E00E94F328802D80939B05A0EFB1E00E94F328802D80932C01A6E0B2E00E9444
S1230680F328802D8093270120E030E0D901AA54BC4F0E94F328802DF901E35DFC4F80836E
S12306A02F5F3F4F2031310589F7A7ECB3E00E94F328802D80933A01A8ECB3E00E94F32851
S12306C0802D80933B01A4EDB3E00E94F328802D8093A705A5EDB3E00E94F328802D80932B
S12306E0A805A6EDB3E00E94F328802D8093A905A7EDB3E00E94F328802D8093AA05A8ED10
S1230700B3E00E94F328802D8093AB05A9EDB3E00E94F328802D8093AC05AAEDB3E00E94F2
S1230720F328802D8093AD05ABEDB3E00E94F328802D8093AE05A8EEB3E00E94F328802D3A
S123074090E090933401809333012091330130913401A9EEB3E00E94F328802D90E0982FE0
S12307608827820F931F9093340180933301AAEEB3E00E94F328802D80939E05ACECB3E06E
S12307800E94F328802D2AE0829FC00111249093B6058093B505A1EDB3E00E94F328802D94
S12307A0829FC00111249093BB058093BA05A2EDB3E00E94F328802D829FC00111249093A3
S12307C0BD058093BC0512BC11BC089580911D0190911E01A2E0B0E0082E0E9400298091B4
S12307E01D0190911E01892F9927A3E0B0E0082E0E9400298091230190912401A4E0B0E07C
S1230800082E0E9400298091230190912401892F9927A5E0B0E0082E0E94002980910001B8
S123082090910101A6E0B0E0082E0E9400298091000190910101892F9927A7E0B0E0082E80
S12308400E94002980911301A8E0B0E0082E0E94002980911201A9E0B0E0082E0E9400294D
S123086012BC11BC089580E0A1EFB1E0082E0E9400298AE0A0EFB1E0082E0E94002980911E
S12308809C05A2EFB1E0082E0E94002984E0A9E5B1E0082E0E94002985E0ACE0B0E0082E55
S12308A00E94002982E3AFE6B1E0082E0E94002924E1A1E7B1E0022E0E94002991E0A0E7CC
S12308C0B1E0092E0E94002988ECA4EFB1E0082E0E940029A5EFB1E0092E0E940029A6EF2C
S12308E0B1E0022E0E9400298AE5A7EFB1E0082E0E94002988EEA8EFB1E0082E0E94002932
S123090083E0A9EFB1E0082E0E94002980912F0190913001ABEFB1E0082E0E940029809176
S12309202F0190913001892F9927ACEFB1E0082E0E9400298091310190913201ADEFB1E0C8
S1230940082E0E9400298091310190913201892F9927AEEFB1E0082E0E9400298091B5048A
S12309609091B604AFEFB1E0082E0E9400298091B5049091B604892F9927A0E0B2E0082E03
S12309800E9400298CEDA7E0B2E0082E0E94002986EEA3E0B2E0082E0E9400292CE132E04C
S12309A088ECD901082E0E9400292F5F3F4F82E02C323807A9F782E2AFE8B1E0082E0E94C5
S12309C0002981E0A6E0B2E0082E0E94002912BC11BC0895CF92DF92EF92FF920F931F9300
S12309E0CF93DF93C0E0D0E0A5E0B2E00E94F328202D30E040E050E0A3EDB3E00E94F3286E
S1230A00602D6E01CC0CDD1C8DE393E0C80ED91EF601E080F18070E080E090E00E9464283F
S1230A2000E010E0A80197010E94642824E630E040E050E00E94B62879018A01CA01B901FF
S1230A4024EF31E040E050E00E94642828EC30E040E050E0E20EF31E041F151FA8019701E3
S1230A600E94B628CA01B9012FEF30E040E050E00E94642825E030E040E050E00E94B628DC
S1230A80E2E0220F331F441F551FEA95D1F7CA01B90124E630E040E050E00E94B628F60189
S1230AA0318320832196C732D10509F09DCFC0E0D0E0A9ECB3E00E94F328202D30E040E03E
S1230AC050E0A3EDB3E00E94F328602D6E01CC0CDD1C8BE893E0C80ED91EF601E080F180BA
S1230AE070E080E090E00E94642800E010E0A80197010E94642824E630E040E050E00E9459
S1230B00B62879018A01CA01B90124EF31E040E050E00E94642828EC30E040E050E0E20E63
S1230B20F31E041F151FA80197010E94B628CA01B9012FEF30E040E050E00E94642825E052
S1230B4030E040E050E00E94B62892E0220F331F441F551F9A95D1F7CA01B90124E630E04F
S1230B6040E050E00E94B628F601318320832196C732D10509F09DCFC0E0D0E0AAECB3E0EF
S1230B800E94F328202D30E040E050E0A3EDB3E00E94F328602D6E01CC0CDD1C89ED93E051
S1230BA0C80ED91EF601E080F18070E080E090E00E94642800E010E0A80197010E9464280F
S1230BC024E630E040E050E00E94B62879018A01CA01B90124EF31E040E050E00E946428FB
S1230BE028EC30E040E050E0E20EF31E041F151FA80197010E94B628CA01B9012FEF30E0B1
S1230C0040E050E00E94642825E030E040E050E00E94B62802E0220F331F441F551F0A9592
S1230C20D1F7CA01B90124E630E040E050E00E94B628F601318320832196C732D10509F0AC
S1230C409DCFC0E0D0E0A4E0B2E00E94F328202D30E040E050E0A3EDB3E00E94F328602DE7
S1230C606E01CC0CDD1C87E294E0C80ED91EF601E080F18070E080E090E00E94642800E090
S1230C8010E0A80197010E94642824E630E040E050E00E94B62879018A01CA01B90124EF6A
S1230CA031E040E050E00E94642828EC30E040E050E0E20EF31E041F151FA80197010E94F2
S1230CC0B628CA01B9012FEF30E040E050E00E94642825E030E040E050E00E94B628B2E08A
S1230CE0220F331F441F551FBA95D1F7CA01B90124E630E040E050E00E94B628F601318365
S1230D0020832196C732D10509F09DCFDF91CF911F910F91FF90EF90DF90CF900895EAE7D7
S1230D20F0E0108280E280937C0080E880BF87EE808311B808950F931F93CF93DF93282F58
S1230D4030E0F901EE0FFF1FEE5FFE4F0081118143E0033F140718F0E2E3F0E04CC053E061
S1230D600F3D150718F0EAE0F0E045C0C0E0D0E087E290E0A901489F9001499F300D589FF9
S1230D80300D1124D901AC0FBD1FAA0FBB1FA35CBC4F8D919C9111978017910730F5FE0189
S1230DA03197E20FF31FEE0FFF1FE35CFC4F20813181608171814D915C91FE01EE0FFF1FB4
S1230DC0EE0FFF1FEC0FFD1F3596201B310BC901880F991F880F991F641B750B820F931FF1
S1230DE00E948F28E60FF71F06C02196C732D10549F6E8ECF0E0CF01DF91CF911F910F916C
S1230E0008950F931F93CF93DF93AC01E0E0F0E0EF01CC0FDD1FDE01AB58BB4F8D919C91CE
S1230E20119748175907C0F56D917C913197EE0FFF1FDF01AB58BB4F8D919C911197681B41
S1230E40790B8D919C91C357DB4F28813981E357FB4F00811181481B590B84E690E0DC0103
S1230E604A9FC0014B9F900D5A9F900D11240E948F28201B310B0190F081E02D629FC001D1
S1230E80639F900D729F900D112464E670E00E948F286E0F7F1F09C03196EA30F10509F025
S1230EA0B7CF6091A1047091A204CB01DF91CF911F910F91089580912A0590912B05282FFA
S1230EC0205527FF0AC08091140190911501BC01660F771F680F791F1EC02F312CF060912A
S1230EE014017091150117C04091140150911501332727FD309588E290E0821B930B9C0119
S1230F00249FC001259F900D349F900D11246AE070E00E948F28CB0108950F931F93CF9331
S1230F20DF93AC018091B8049091B9044817590718F4E0EFF0E057C08091D4049091D5047F
S1230F408417950718F4E0E0F0E04DC0E1E0F0E0EF01CC0FDD1FDE01A854BB4F8D919C9125
S1230F60119748175907C0F56D917C913197EE0FFF1FDF01A854BB4F8D919C911197681B07
S1230F80790B8D919C91EA52FB4F20813181CA52DB4F08811981481B590B84E690E0DC01BE
S1230FA04A9FC0014B9F900D5A9F900D11240E948F28201B310B0190F081E02D629FC00190
S1230FC0639F900D729F900D112464E670E00E948F28E61BF70B07C03196EE30F10509F0FA
S1230FE0B7CFEEEFF0E0CF01DF91CF911F910F9108958091B305882359F08CED95E090935F
S12310003601809335011092C8051092C7052AC08091B305882349F08CED95E09093360190
S12310208093350184E690E019C08091B305882349F08CED95E090933601809335018AEFF9
S123104090E00CC08091B305882361F08CED95E0909336018093350184EF91E09093C80526
S12310608093C705F89480919705909198058A5A9A4AC1F0809197059091980585559545FE
S123108089F0789480912606909127068064909327068093260684EF91E090933601809378
S12310A035010AC0789480912606909127068F7B9093270680932606F894809199059091A0
S12310C09A058F3F89F0789480912606909127068068909327068093260684EF91E0909311
S12310E03601809335010AC0789480912606909127068F779093270680932606809135012F
S123110090913601892B99F12F9A2091C7053091C8052115310511F42F9A16C08091C50576
S12311209091C605029780F485B1881F8827881F809587958827879595B19F77982B95B916
S12311403093C6052093C5058091C5059091C60501979093C6058093C505809135019091EE
S123116036010197909336018093350108952F981092C8051092C7050895809126069091BD
S123118027069F779093270680932606809100019091010197FD44C08091280580FF32C0FD
S12311A020918F053091900580911F01909120018C599F4F8217930720F461E070E040E84A
S12311C032C020918F053091900580911F019091200149978217930720F461E070E048E02B
S12311E022C020918F053091900580911F0190912001845690408217930790F461E070E009
S123120044E011C020918F053091900580911F01909120018217930718F460E070E802C02E
S123122060E070E040E02091260630912706CB019927869597958827822B932B90932706F2
S1231240809326062091260630912706CB0180709078822B932B9093270680932606209111
S12312603805309139058091380190E08217930734F480913801882311F0606148608091A9
S1231280A80520913A0530913B0590E08F5B9F4F8217930774F48091A805882351F060625D
S12312A080918F0590919005895B9B40A0F0446012C08091A80520913A0530913B0590E0EB
S12312C0C296821793073CF48091A805882319F0606251E001C050E08091A7052091400546
S12312E03091410590E0C296821793076CF48091A705882349F0606480918F0590919005C8
S1231300855C994008F044608091A90520913E0530913F0590E0C2968217930734F4809187
S1231320A905882311F0606844608091AA0520913C0530913D0590E0C2968217930734F40B
S12313408091AA05882311F0606844608091AB05209142053091430590E0880F991F821797
S1231360930734F48091AB05882311F0606844608091AC05209144053091450590E0880F00
S1231380991F8217930734F48091AC05882311F0606844608091AD05209146053091470590
S12313A090E0880F991F8217930734F48091AD05882311F0606844608091AE052091480572
S12313C03091490590E0880F991F8217930734F48091AE05882311F060684460552321F07B
S12313E082E380938B0502C010928B05189906C07093B1056093B0054093B2054093B30500
S12314000895809100019091010193FF1FC11A9B06C08091B9058F5F8093B90502C0109217
S1231420B9058091B905853108F454C01092B40520918F05309190058091B5049091B604BA
S12314408217930778F48091B0059091B10582609093B1058093B0058091B2058860809306
S1231460B20509C08091B0059091B1058D7F9093B1058093B0058091280583FF16C08091F7
S12314808F0590919005815D974078F08091B0059091B10584609093B1058093B0058091AE
S12314A0B20582608093B20509C08091B0059091B1058B7F9093B1058093B0058091B505E9
S12314C09091B6059093B8058093B70584E38093B905B1C08091B7059091B805892B09F478
S12314E05DC08091B7059091B80501979093B8058093B7058091B405823099F0833030F4FD
S1231500882351F0813009F096C019C08330A9F1843009F090C031C01092B8051092B7050A
S12315208AC08091B0059091B10584609093B1058093B0058091B20582608093B205209116
S12315408F05309190058091B5049091B6048217930768F48091B0059091B10582609093C7
S1231560B1058093B0058091B205886059C08091B0059091B1058D7F0CC09091CE058091A6
S1231580B704891708F440C08091B0059091B1058B7F9093B1058093B0054DC04E9B20C0D2
S12315A080918F05909190058D5D9540C8F08091C3059091C40501969093C4058093C30534
S12315C02091BA053091BB0528173907A0F58091BC059091BD059093C2058093C10514C0B6
S12315E02091C1053091C20521153105E1F080918F05909190058D5D9540A8F02150304018
S12316003093C2052093C1058091B0059091B10584609093B1058093B0058091B2058260F7
S12316208093B20508C01092C4051092C3051092C2051092C1058091B20581FF07C080914E
S12316402E0180FF03C084E68093F00508959C018091280584FF1BC022533040C901F3E04B
S1231660880F991FFA95E1F7220F331F280F391F2455354F442737FD4095542F60E579E705
S123168084E090E00E94D828822F90E008958091280585FD03C084E690E008952253304033
S12316A0C90173E0880F991F7A95E1F7220F331F280F391F2455354F442737FD4095542FCD
S12316C060E579E784E090E00E94D8282C592695822F90E00895A89582E50E94AA2783E172
S12316E00E94AA2780918F0590919005892F99270E94AA2780918F05909190050E94AA275F
S123170080914005909141050E94AA2780913A0590913B050E94AA2780912A0590912B05E0
S12317200E94AA2780913805909139050E94AA2780913605909137050E94AA2780913205AE
S1231740909133050E94AA2780919505909196056091180170E00E948F28CB010E94AA2760
S1231760809194050E94AA27809193050E94AA2720912606309127068091F6059091F70538
S1231780E3E096958795EA95E1F78170232F3327822B0E94AA2780912606909127060E94FA
S12317A0AA278091570680950E94AA27809148060E94AA2780913005909131050E94AA277C
S12317C08091F8059091F905969587950E94AA272091CB0530E0220F331FF901E65CFA4F85
S12317E080819181892F990F990BB3E0220F331FBA95E1F7822B0E94AA27E091CB05F0E060
S1231800EE0FFF1FE65CFA4F808191810E94AA278DEA0E94AA278091CB058F5F8093CB05FC
S1231820883010F01092CB050895CF92DF92EF92FF920F931F93CF93DF93A89588E10FB666
S1231840F89480936000109260000FBE0E94F627882309F495C50E9487279093CA058093A0
S1231860C9058136910509F486C08236910508F041C08D34910509F4E1C18E349105E8F495
S12318808134910509F49CC08234910568F48932910509F4B1C48433910509F458C5883214
S12318A0910509F06BC585C48534910509F4C1C08634910509F062C545C18335910509F48E
S12318C0EDC48435910548F48035910509F433C38235910509F052C5AAC38735910509F471
S12318E0A1C38835910509F432C48535910509F045C5E5C38936910509F4CEC28A36910507
S1231900E8F48436910509F43BC58536910548F48236910509F495C28336910509F02EC530
S123192093C28636910509F4EBC08636910508F4F8C18736910509F021C5D5C28037910537
S123194009F4FEC28137910548F48D36910509F434C18F36910509F011C511C4893791059C
S123196009F46DC48A37910509F471C28837910509F004C56CC281E60E94AA2780EA0E9483
S1231980AA271092CA051092C9050EC0ED5BFE4F80810E94AA278091C9059091CA05019654
S12319A09093CA058093C905E091C905F091CA05E03AF10558F382E30E94FB268EE9DEC425
S12319C01092CA051092C905C0E0D0E00E94F627882341F1C091C905D091CA05C03AD10517
S12319E089F40E9487279093CA058093C9058E3B910519F4C6E1DAEF15C08091C9050E9411
S1231A00AA27FBCF0E948727CD5BDE4F88838091C9059091CA0501969093CA058093C9053E
S1231A20C0E0D0E021964AEFC030D40708F0A8C4CDCFC0E0D0E00E94F627882309F459C0C7
S1231A400E9487278A3B910509F09AC488E10FB6F89480936000109260000FBE1092CA0513
S1231A601092C9053EC0885B0E94AA278DEF0E94AA272091C9053091CA058AEF90E0289FF0
S1231A80E001299FD00D389FD00D112407C0DE010E94F328802D0E94AA2721962091C9051A
S1231AA03091CA052F5F3F4F8AEF90E0AC01249FC001259F900D349F900D11242150304075
S1231AC0C817D90720F3822F885B80950E94AA278091C9059091CA0501969093CA058093A9
S1231AE0C9058091C9059091CA058430910508F4BACF21965AEFC030D50708F041C49BCF43
S1231B0086E60E94AA2780EA0E94AA271092CA051092C9050EC0ED51FE4F80810E94AA2757
S1231B208091C9059091CA0501969093CA058093C905E091C905F091CA05E03AF10558F37E
S1231B4089E91CC41092CA051092C90500E010E00E94F627882349F1C091C905D091CA058B
S1231B60C03AD10591F40E9487279093CA058093C905893B910519F406E11AEF16C0E0914B
S1231B80BF05F091C005099510C00E948727CD51DE4F88838091C9059091CA05019690939A
S1231BA0CA058093C90500E010E00F5F1F4F8AEF0030180708F0E4C3CBCF8DE60E94AA27DE
S1231BC089E00E94AA2780911D0190911E010E94AA2780911D0190911E01892F99270E94BA
S1231BE0AA2780912301909124010E94AA278091230190912401892F99270E94AA278091AB
S1231C000001909101010E94AA278091000190910101892F99270E94AA27809113010E9442
S1231C20AA27809112010E94AA27AAE0B0E00E94F328802D0E94AA2782E9A0C31092CA0502
S1231C401092C905C0E0D0E00E94F6278A3008F461C00E94872790931E0180931D010091D6
S1231C601D0110911E010E948727982F8827800F911F90931E0180931D010E948727909397
S1231C8024018093230100912301109124010E948727982F8827800F911F90932401809309
S1231CA023010E948727909301018093000100910001109101010E948727982F8827800FE9
S1231CC0911F90930101809300010E948727809313010E948727809312010E948727AAE050
S1231CE0B0E0082E0E9400290E94D0210E948727823B910551F40E94E603E091BF05F09193
S1231D00C0050995CFE6DAEF05C0E091BF05F091C005099521964AEFC030D40708F030C35A
S1231D2093CF85E60E94AA2783E10E94AA271092CA051092C9050EC0ED5DFC4F80810E94A1
S1231D40AA278091C9059091CA0501969093CA058093C905E091C905F091CA05EA30F105D6
S1231D6058F3809119010E94AA2780911B010E94AA2783E00E94FC26809128010E94AA2702
S1231D80809129010E94AA2780912A010E94AA2780912B010E94AA278091140190911501D5
S1231DA066E070E00E948F28CB010E94AA27809125010E94AA27AEE6B1E00E94F328802DB8
S1231DC00E94AA278AE90E94AA278CE60E94AA2784E10E94AA271092CA051092C9050EC03A
S1231DE0E550FA4F80810E94AA278091C9059091CA0501969093CA058093C905E091C90575
S1231E00F091CA05EA30F10558F31092CA051092C9050EC0E550FA4F80890E94AA27809159
S1231E20C9059091CA0501969093CA058093C905E091C905F091CA05EA30F10558F383E920
S1231E409DC20E9486009CC20E94C10099C20E946B0B96C20E948727C82FD0E00E94872724
S1231E60C817D90709F08CC20E9487278C019093CA058093C9050E9487270817190709F020
S1231E807FC20E9487278639910509F079C28091C905CD5BDE4F4DC00E94F6278530D0F6A9
S1231EA0FBCF0E948727C82FD0E00E948727C817D90709F065C20E9487278C019093CA055F
S1231EC08093C9050E9487270817190709F058C20E9487278839910509F052C28091C905E8
S1231EE0CD51DE4F26C00E94F6278530D0F6FBCF0E948727C82FD0E00E948727C817D907A3
S1231F0009F03EC20E9487278C019093CA058093C9050E9487270817190709F031C20E94F7
S1231F2087278F3A910509F02BC28091C905CD57DD4F888325C20E94F6278530C8F6FBCF8D
S1231F40C0E0D0E00E94F627823080F10E9487270E9487278F38910509F012C21092CA0510
S1231F601092C9051CC0ED57FD4F108180E70E94AA2782E00E94AA278091C9050E94AA27EF
S1231F80812F0E94AA278FE80E94AA278091C9059091CA0501969093CA058093C905E09186
S1231FA0C905F091CA05E03AF105E8F221965AEFC030D50709F4E4C1C5CF0E9487278C0136
S1231FC00E948727D82FCC27C00FD11F0E9487278C019093CA058093C9050E9487270817D5
S1231FE0190709F0CDC10E948727883A9105A9F4DE010E94FB28E0708091C9059091CA052E
S1232000E82BF92BF093CA05E093C905DE010F010E940C2912BC11BCB3C1E091BF05F09167
S1232020C00509950E94F627853038F6FBCFCC24DD240E94F6278330C0F10E9487278C01DC
S12320400E948727EC010E9487278D3A910509F097C1FC2EEE24E00EF11ED7010E94F32873
S1232060802D90E0D70111960E94F328002D10E0102F0027080F191F84E50E94AA2784E0F1
S12320800E94AA27802F0E94AA278E2D0E94AA27EF2CFF248E2D0E94AA27012F1127802FF6
S12320A00E94AA278BEA0E94AA270894C11CD11C80E0C8168AEFD80609F462C1BACFCC242D
S12320C0DD240E94F6278330C0F10E9487278C010E948727EC010E9487278A3A910509F01B
S12320E04FC1FC2EEE24E00EF11ED7010E94F328802D90E0D70111960E94F328002D10E088
S1232100102F0027080F191F85E50E94AA2784E00E94AA27802F0E94AA27012F1127802F19
S12321200E94AA278E2D0E94AA27EF2CFF248E2D0E94AA278AEA0E94AA270894C11CD11C41
S123214040E0C4164AEFD40609F41AC1BACFC0E0D0E00E94F627882359F00E948727873AF9
S1232160910509F00DC1E091BF05F091C005099521965AEFC030D50709F402C1EACFC0E000
S1232180D0E00E94F627882369F00E9487278039910509F0F5C00E94FD00E091BF05F09126
S12321A0C005099521968AEFC030D80709F4E8C0E8CFC0E0D0E00E94F6278823B1F00E9460
S12321C08727873D910509F0DBC08091360590913705ADE6B1E0082E0E94002912BC11BCF6
S12321E0E091BF05F091C005099521964AEFC030D40709F4C5C0DFCFC0E0D0E00E94F627C8
S12322008823B1F00E948727863D910509F0B8C08091360590913705AEE6B1E0082E0E94AE
S1232220002912BC11BCE091BF05F091C005099521965AEFC030D50709F4A2C0DFCFC0E044
S1232240D0E00E94F627823010F10E948727892B09F096C00E94872786389105C1F489E73C
S12322600E94AA2785E00E94AA278FEC0E94AA278FE30E94AA278DE00E94AA2783E40E9453
S1232280AA278CE00E94AA2786E80E94AA2721968AEFC030D80709F473C0D3CFC0E0D0E088
S12322A00E94F627823008F44CC00E948727892B09F047C00E9487278C3A910509F060C0D8
S12322C083E50E94AA2788E00E94AA2780919705909198050E94AA278091970590919805FB
S12322E0892F99270E94AA2780912406909125060E94AA278091240690912506892F9927F6
S12323000E94AA2780911F06909120060E94AA2780911F0690912006892F99270E94AA27EE
S123232080915B0690915C060E94AA2780915B0690915C06892F99270E94AA278CEA0E9439
S1232340AA2721964AEFC030D407D1F0A9CFC0E0D0E00E94F627823058F00E948727892BA7
S123236079F40E9487278B3C910511F40E94110121965AEFC030D50719F0EBCF0E94AA2784
S1232380A895DF91CF911F910F91FF90EF90DF90CF9008950F931F93CF93DF93109227066C
S12323A0109226060E94F3263D9A3E9A3C9A459A469A449A3F9A479A389840983998419862
S12323C03A9842983B984398389839983A983B9854985C9855985D9854985598239A269A41
S12323E0279A2B9A2E982F98259A249A5398529822985698219820980E94FE26AAE5B1E075
S12324000E94F328802D80939D050E947B210E94D0210E94E1260E948F060E94EA042B9A93
S12324202E98A7E0B0E00E94F328802D12BC11BC85FF9BC080910001909101019F7D909363
S12324400101809300010E94E6030E9433040E94C1000E9486000E94FD0086E0AAE0B0E054
S1232460082E0E94002989E1ABE0B0E0082E0E9400298EE1ACE0B0E0082E0E940029AEE0B7
S1232480B0E0082E0E94002920E030E0F901ED5DFC4F8081D901A25ABE4F082E0E94002923
S12324A02F5F3F4F2A30310589F780912801A9E6B1E0082E0E94002980912901AAE6B1E035
S12324C0082E0E94002980912A01ABE6B1E0082E0E94002980912B01ACE6B1E0082E0E9460
S12324E0002920E030E0F901E550FA4F8081D901AE58BE4F082E0E9400292F5F3F4F2A30C2
S1232500310589F720E030E0F901E550FA4F8089D901A458BE4F082E0E9400292F5F3F4F70
S12325202A30310589F780911E06A1E7B1E0082E0E940029809114019091150166E070E045
S12325400E948F28ADE0B0E0062E0E94002984E1ADE6B1E0082E0E94002981EEAEE6B1E0E4
S1232560082E0E94002912BC11BC0E94E8000E9411010E949A000E9461008091000190910B
S1232580010185FD07C080916F008B7F80936F00459A469A80912701882311F480E801C00F
S12325A080E4809339011092290580911401909115018D5A9D4030F08CEA9DE09093150129
S12325C08093140110928C0586B3866086BB78948AEA0E94AA2780E00E94AA2785E50E946A
S12325E0AA2783B18695817080939F0580916E00836080936E002B9A2E9AA89580918F05BD
S1232600909190058E37910570F180918C05882351F580912606909127069F7E90932706B9
S12326208093260680916F00856080936F0080916E00836080936E002B9A81E080938C05C3
S12326408091260690912706806290932706809326068091260690912706906290932706AD
S12326608093260649C080918C05813009F044C080918F05909190058635910508F03CC01E
S123268080916F008D7F80936F00809170008C7F8093700080916F008B7F80936F008091FC
S12326A06E00836080936E0080912606909127068F7D9093270680932606809126069091C0
S12326C02706877F9093270680932606389839983A983B9854985598459A469A449A1092D6
S12326E08C0580912606909127069F7D909327068093260610928A0580918C058130F9F49E
S123270080918A058823C1F080916F00826080936F008091700083608093700080916E006F
S1232720836080936E008091260690912706886090932706809326062B9A2E9A14C010922C
S12327408A05459A469A449A10928A051092B3001092960510929505809141019091420193
S1232760892B09F42B9880912905833009F4DCC0843018F4882371F077C0853009F4E7C1F9
S1232780853008F442C1863009F4CDC1873009F093C21CC280918D0590918E0585369105B5
S12327A008F48DC2E0912905F0E080917800909179008C7F65E070E00E948F28EE0FFF1F24
S12327C0E659FA4F7183608380912905C82FD0E0E0912905F0E0EE0FFF1FE65DFA4F808199
S12327E09181E0912905F0E0EE0FFF1FE659FA4F20813181880F991F880F991F820F931F7D
S1232800880F991F6AE070E00E948F28CC0FDD1FC65DDA4F7983688310928E0510928D05FF
S1232820809129058F5F8093290580912905806480937C000E94150C0E945B079093170172
S1232840809316018091410190914201892B09F431C280914101909142010197909342013A
S1232860809341012B9A26C280918D0590918E058536910508F423C2909129054091AF05F5
S1232880842F83708450990F990F980FE92FF0E0EE0FFF1FEE5FFE4F8081918120917800EA
S12328A030917900820F931F969587959183808310928E0510928D05A89580912905C42F61
S12328C0D0E08130D1F48E01085F1F4F842F0E949B06000F111F065D1A4FF8019183808359
S12328E08091AF058823A9F480913A0590913B050E94270B80934C060CC08081918162E0BC
S123290070E00E94A328CC0FDD1FCE5BDA4F79836883809129058F5F809329058091290539
S1232920806480937C00CBC180918D0590918E058536910508F4C3C1E0912905F0E08091EC
S12329407800909179009695879596958795EE0FFF1FE659FA4F9183808380912905C82FE3
S1232960D0E0E0912905F0E0EE0FFF1FE65DFA4F80819181E0912905F0E0EE0FFF1FE659B1
S1232980FA4F20813181880F991F880F991F820F931F880F991F6AE070E00E948F28CC0F99
S12329A0DD1FC65DDA4F7983688310928E0510928D05809129058F5F8093290580912905CE
S12329C090913901892B80937C000E94150CA8958091AF058F5F8093AF05843010F0109285
S12329E0AF052091AF05922F91709295990F907E85B18F7D892B85B9220F220F220F2071C3
S1232A0085B18F7E822B85B95AC180918D0590918E058159914008F452C180912701882374
S1232A2029F1E0912905F0E080917800909179009695879596958795EE0FFF1FE659FA4FB5
S1232A4091838083A0912905B0E0E0912905F0E0EE0FFF1FE659FA4F80819181AA0FBB1FB4
S1232A60A65DBA4F11969C938E933EC0E0912905F0E08091780090917900EE0FFF1FE65965
S1232A80FA4F9183808380912905C82FD0E0E0912905F0E0EE0FFF1FE65DFA4F00811181C3
S1232AA0E0912905F0E0EE0FFF1FE659FA4F808191810E948D079C01220F331F280F391F08
S1232AC0C80143E0880F991F4A95E1F7801B910B820F931F6AE070E00E948F28CC0FDD1FBC
S1232AE0C65DDA4F7983688310928E0510928D05809129058F5F80932905809129058068A1
S1232B0080937C0020919F0583B18695817030E090E02817390709F4CDC0E091BF05F0914E
S1232B20C0050995C7C080918D0590918E058536910508F4C4C0E0912905F0E08091780087
S1232B409091790096958795969587950FC080918D0590918E05893C910508F4B0C0E091EB
S1232B602905F0E08091780090917900EE0FFF1FE659FA4F91838083A0912905B0E0E09116
S1232B802905F0E0EE0FFF1FE65DFA4F20813181E0912905F0E0EE0FFF1FE659FA4F808126
S1232BA09181820F931F96958795AA0FBB1FA65DBA4F11969C938E9310928E0510928D0576
S1232BC0809129058F5F809329056DC080918D0590918E058536910508F471C0E0912905E2
S1232BE0F0E08091780090917900969587959695879590E0EE0FFF1FE659FA4F9183808326
S1232C00E0912905F0E0EE0FFF1FE65DFA4F80819181843691050CF5A0912905B0E0E091D6
S1232C202905F0E0EE0FFF1FE65DFA4F40815181E0912905F0E0EE0FFF1FE659FA4F2081A5
S1232C403181CA01880F991F840F951F820F931F969587959695879519C0A0912905B0E0C4
S1232C60E0912905F0E0EE0FFF1FE65DFA4F20813181E0912905F0E0EE0FFF1FE659FA4FD5
S1232C8080819181820F931F96958795AA0FBB1FA65DBA4F11969C938E9310928E05109226
S1232CA08D051092290580912905806480937C000E94150CA89503C081E080932905809186
S1232CC08D0590918E05019690938E0580938D0580918F05909190058752924008F45BC09B
S1232CE080914A068F5F80934A0690914A0680914B06981708F452C010924A06809138054E
S1232D0090913905E0916106FF27E7FDF095E85DF94F208130E08217930754F480914806D1
S1232D20843634F48091480690914906890F17C08091380590913905E0916106FF27E7FDE0
S1232D40F095E85DF94F208130E0821793074CF08091480682302CF08091480681508093CD
S1232D60480680914806E0916106FF27E7FDF095E85DF94F2089992787FD909530E028174D
S1232D80390764F4E0916106FF27E7FDF095E85DF94F808901C081E08093480680918F0572
S1232DA0909190058739910508F46DC020913605309137058091250190E0499628173907EC
S1232DC00CF061C08091F2059091F30501969093F3058093F2052091F2053091F305809183
S1232DE0F4059091F5052817390708F440C01092F3051092F20520918F0530919005809161
S1232E00EC059091ED050A972817390730F49091F0058091F105890F15C020918F053091D6
S1232E2090058091EC059091ED0549968217930758F49091F0058091EF05891728F480919E
S1232E40F00581508093F0059091F0058091EE05891718F48091EE0508C09091F0058091E7
S1232E60EF05981720F48091EF058093F00580918F05909190058A58924038F48091EE054B
S1232E808093F00502C01092F0058091280582FF4FC080918F0590919005855F914008F4F3
S1232EA047C080918F0590919005805D974008F03FC020913605309137058091250190E071
S1232EC0059628173907A4F520913605309137058091A20590E00196821793074CF1809112
S1232EE0A3059091A405A091A505B091A6050196A11DB11D8093A3059093A405A093A5050E
S1232F00B093A6058091A3059091A405A091A505B091A6058158994AA340B04010F181E084
S1232F208093A1058091260690912706916015C080913605909137058093A2051092A305D6
S1232F401092A4051092A5051092A6051092A10580912606909127069E7F90932706809336
S1232F602606809100019091010192FF27C020918F053091900580912F01909130018217AD
S1232F809307E0F420918F053091900580913101909132012817390788F4209136053091E5
S1232FA037058091250190E005962817390734F48091260690912706946005C08091260667
S1232FC0909127069B7F90932706809326060E94BD080E94010A0E94F9078091000190910D
S1232FE0010180FF67C080912E0180FF11C08091EB05883C28F08091F0058823B9F418C082
S12330009091F0058091EB058695891790F010C080912E0182FF0DC08091EB05883C48F0FF
S1233020809126069091270696FF02C0549A01C0549880912E0184FF16C08091EB05883CB1
S123304028F08091480618165CF12CC0209148068091EB05332727FD3095869590E0821727
S123306093070CF11FC080912E0186FF1CC08091EB05883CC0F020918F0530919005809114
S12330803301909134018217930760F4209138053091390580919E0590E08217930714F4CF
S12330A0559A01C055988091EB05883C28F01092EB0502C0549855988091EB058F5F809363
S12330C0EB059ACA1F920F920FB60F9211248F939F93809162068F5F8093620680916206FC
S12330E0882309F447C080912606909127069061909327068093260610928C0580912606A2
S1233100909127069F7D909327068093260680916F008B7F80936F0080916F008D7F809307
S12331206F00809170008C7F8093700080916E00836080936E00459A469A449A8091260650
S1233140909127068F7D90932706809326068091260690912706877F909327068093260662
S1233160389839983A983B98549855981092900510928F0578949F918F910F900FBE0F9058
S12331801F90189520915F063091600680918400909185002817390760F580915106863065
S12331A0A1F48091990590919A05880F991F90939A05809399058091990590919A058160F5
S12331C090939A058093990504C010929A051092990581E0809351068091F4049091F50445
S12331E09093F7048093F6041092F5041092F40405C0809151068F5F809351068091840051
S1233200909185009093600680935F0608951F920F920FB60F9211248F939F938091F4041C
S12332209091F50401969093F5048093F4049F918F910F900FBE0F901F901895282F809193
S123324026069091270693FD0BC0223031F0233031F0213029F4459808954698089544986F
S123326008951F938091E405882309F45CC08091E4058130A1F4459A1092E4058091F4048A
S12332809091F50490936B0680936A0680918F05909190058559914198F182E02FC0809103
S12332A0E4058230A1F4469A1092E4058091F4049091F504909356068093550680918F05BA
S12332C09091900585599141D8F083E017C08091E4058330A9F4449A1092E4058091F404C6
S12332E09091F504909364068093630680918F05909190058559914118F081E00E941E195A
S123330080911F0690912006892B69F180915D06882349F180911F069091200690938B009A
S123332080938A0020C080915D068823E1F010915D06113041F010915D06123021F01091AE
S12333405D06133031F480915D060E941E191093E40580915B0690915C0690938B0080930F
S12333608A0010925D061F9108951F920F920FB60F9211242F933F934F935F936F937F9304
S12333808F939F93AF93BF93EF93FF930E9431192B9A7894FF91EF91BF91AF919F918F9180
S12333A07F916F915F914F913F912F910F900FBE0F901F9018951F920F920FB60F92112445
S12333C08F939F93F89480915206882309F486C08091B0059091B10597FD80C0809113011C
S12333E08095809357068091570690911B068C59891B809357069091FA05943029F19530D8
S123340040F4923051F19330B8F4913009F058C009C09731C1F1933609F441C09E3009F05E
S12334204FC023C0809157068093B20084E08093B100389A83E050C08091570686BD83E0E2
S123344085BD3A9A84E048C0809157068093B2009093B1003B9A82E03FC08091570686BDF8
S123346083E085BD399A81E037C081E080931105809157068093B20084E08093B100389AC1
S12334803B9A87E129C081E0809312058091570686BD83E085BD399A3A9A8EE01DC081E0CE
S12334A080931105809157068093B20084E08093B100389A3B9A3A9A399A9093FA050EC046
S12334C0809157068093B20084E08093B100389A3B9A3A9A399A83E68093FA0578949F9188
S12334E08F910F900FBE0F901F901895CF93DF93EC0180919C05E7E0F0E0E81BF109EE0F3D
S1233500FF1FE65DFA4F8081918120919B05821B282F30E080912C0190E0880F991F880F01
S1233520991FAC01429FC001439F900D529F900D112464E670E00E948F286436710520F02B
S123354083E680935E0602C060935E0680915E066AE00E94832880934F0680914F068A30DA
S12335602CF089E080934F0680934F0680918F0590919005885E934008F0B3C010924D067E
S12335808FEF8093610680914F06992787FD909564E0880F991F6A95E1F78093930580913A
S12335A08F059091900564E670E00E948F28655060935A0680918F0590919005845F9140B3
S12335C060F410925A06E0915A06FF27E7FDF095E45CFE4F808190E0A3C080915A068430AB
S12335E0D9F5E0919305F0E0ED5BFE4F2081E0915A06FF27E7FDF095E45CFE4F6081E091AB
S12336005A06FF27E7FDF095E45CFE4F808190E09093F9058093F805E091F805F091F9059B
S123362080918F059091900540915A0630E0220F331F261B3109845F91406CE94602A001FA
S12336401124840F951FAC01249FC001259F900D349F900D11243AC0E0915A06FF27E7FDDE
S1233660F095E35CFE4F6081E0915A06FF27E7FDF095E45CFE4F4081E0915A06FF27E7FDCB
S1233680F095E45CFE4F808190E09093F9058093F805E091F805F091F90580918F059091BF
S12336A0900520915A0670E0641B7109845F91404CE9240290011124820F931F9C01629F61
S12336C0C001639F900D729F900D112464E670E00E948F28E60FF71FF093F905E093F805B4
S12336E0C7C080918F0590919005875F9242E8F086E980934D068FE08093610680914F062E
S1233700909161068295807F890F80939305E0919305F0E0ED5BFE4F808190E0880F991F96
S12337209093F9058093F805A3C080918F0590919005885E934062E370E00E948F286093FC
S12337404D0680914D066AE00E9483288093610680914F06909161068295807F890F8093EE
S12337609305E0919305F0E0ED5BFE4F808190E0880F991F9093F9058093F80580916106D6
S123378087FD39C0809161068F30ACF5E0919305F0E0EC5BFE4F8081E0919305F0E0ED5B41
S12337A0FE4F6081E091F805F091F90520914D0640916106861B880F992787FD909530E0FD
S12337C06AE04602A0011124241B350BAC01429FC001439F900D529F900D11246AE070E0D3
S12337E00E94A328772767FD70956E0F7F1F7093F9056093F80580914F0687FD39C0809151
S12338004F068930ACF5E0919305F0E0ED5AFE4F8081E0919305F0E0ED5BFE4F6081E091C7
S1233820F805F091F90520915E0640914F06861B880F992787FD909530E06AE04602A001E9
S12338401124241B350BAC01429FC001439F900D529F900D11246AE070E00E94A32877277A
S123386067FD70956E0F7F1F7093F9056093F8058091260690912706977F909327068093CB
S123388026068091F6059091F705877F9093F7058093F6058091B205882309F458C0809103
S12338A0B20588233CF18091B205883088F08091500690E083709070892B09F448C08091E9
S12338C0500667E00E948328992309F440C012C08091B2058430C0F08091500690E0837079
S12338E09070892B39F08091500667E00E948328992369F58091260690912706986090932C
S123390027068093260623C08091B205823050F08091F6059091F70588609093F705809357
S1233920F60515C08091B205882389F08091F8059091F9058739910550F08091F8059091D5
S1233940F9058C5890409093F9058093F805809150068F5F809350064091CE05445645310E
S12339600CF044E12091F8053091F9058091120190918B05285B3F4F280F311D291B3109CC
S1233980842F4C3E0CF48CEE992787FD9095280F391F3093CD052093CC058091CC05909158
S12339A0CD058D5B92402CF06CEB72E080E090E015C08091CC059091CD0505972CF465E037
S12339C070E080E090E00AC08091CC059091CD059C01B901882777FD8095982F2091910587
S12339E0309192052C0F3D1F40E050E00E94642820EB34E040E050E00E94B628C21BD30BAC
S1233A00CE01DF91CF910895A0E0B0E0BC01CD0128E532E040E050E00E94642820EB34E00F
S1233A2040E050E00E94B628DA01C90108950F931F93CF93DF9380910A0590910B059093D4
S1233A4069068093680680910A0590910B05499708F456C280916206882349F088EE9DEFCE
S1233A6090930F0580930E051092620653C080918F059091900540910E0550910F05895BB0
S1233A809B40C0F0E0919105F091920520910A0530910B058091F80490E0241B350BAC013E
S1233AA0429FC001439F900D529F900D112464E170E017C0E0919105F091920520910A05D3
S1233AC030910B058091F80490E0241B350BAC01429FC001439F900D529F900D11246EE135
S1233AE070E00E94A328CB018E0F9F1F62E070E00E94A32870939205609391051092920583
S1233B001092910580910A0590910B0590930F0580930E0580918A05893628F480918A05A0
S1233B208F5F80938A0580918F0590919005C0910E05D0910F05D0932506C0932406209101
S1233B4024063091250600910C0510910D0540E050E060E070E489E191E00E94D828CA01CA
S1233B60B90124E130E040E050E00E94642820EC30E0A901049F9001059F300D149F300D29
S1233B8011242050324040E050E00E94B6283093900520938F0580918F0590919005815D62
S1233BA0974010F0E89801C0E89A2091DB053091DC054091D9055091DA05C901880F991FAC
S1233BC0820F931F840F951F96958795969587959093DC058093DB058091D7059091D805E7
S1233BE09093DA058093D9058091D5059091D6059093D8058093D7058091D3059091D40515
S1233C009093D6058093D5058091D1059091D2059093D4058093D3058091CF059091D00514
S1233C209093D2058093D10580918F05909190059093D0058093CF0580918F059091900508
S1233C408D5D9540B8F08091CE054091CF055091D0052091DB053091DC0590E0821B930BDC
S1233C60840F951F9695879596958795855B8093CE050FC084E68093CE05809191059091BE
S1233C80920564E070E00E94A32870939205609391051092620680918F05909190058C5222
S1233CA09140A0F580910C0590910D05039771F580915106813051F584E090E090930D05DD
S1233CC080930C0580910C0590910D0580688093810080918400909185009695879596953E
S1233CE087959093850080938400D695C795D695C795D0930F05C0930E058091240690919E
S1233D00250696958795969587953AC080918F0590919005875B9340B8F180910C059091F0
S1233D200D05049789F580915106813069F583E090E090930D0580930C0580910C0590916E
S1233D400D058068809381008091840090918500880F991F880F991F9093850080938400B9
S1233D60CC0FDD1FCC0FDD1FD0930F05C0930E058091240690912506880F991F880F991F8F
S1233D80909325068093240680912406909125060E94761A90935C0680935B068091F605D6
S1233DA09091F70583FF3AC0E091E505F091E605CF0183709070892B99F4209124063091FF
S1233DC0250680912406909125066AE070E00E948F28261B370B30935C0620935B0618C0A6
S1233DE020913A01809124069091250668E270E00E948F2830E0629FC001639F900D729FD7
S1233E00900D11248C599F4F90935C0680935B063196F093E605E093E50504C01092E6051D
S1233E201092E50580918F05909190058A58924038F080912A0590912B058E3691053CF4A0
S1233E408CE291E0909366068093650604C0109266061092650680915B0690915C062091ED
S1233E601601309117014091650650916606821B930B841B950B9093540680935306809151
S1233E8053069091540697FF20C08091530690915406209124063091250640915B06509115
S1233EA05C06820F931F8417950778F4209124063091250680915B0690915C06821B930BBF
S1233EC044969093540680935306F89480915106833011F48EE005C080915106843081F4AB
S1233EE087E18093FA0580912406909125060E94041D909389008093880081E080935206E7
S1233F007894DF91CF911F910F9108951F920F920FB60F9211242F933F934F935F936F937D
S1233F207F938F939F93AF93BF93EF93FF934B9919C00E94171D0E94C21880919705909192
S1233F409805880F991F909398058093970580919705909198058160909398058093970547
S1233F604798B6C1209184003091850080910A0590910B05969587952817390770F48091E0
S1233F808F0590919005815D974038F081E090E090939805809397059BC18091F60590912D
S1233FA0F70583FFA2C0809184009091850090930B0580930A05109285001092840080912F
S1233FC0970590919805880F991F9093980580939705479A20913A01809124069091250671
S1233FE068E270E00E948F2830E0629FC001639F900D729F900D11248C599F4F90935C061E
S123400080935B0680918F05909190058051974208F057C0809126069091270693FD51C0E8
S123402080915B0690915C0690938B0080938A0020912406309125068091240690912506EE
S12340409695879596958795281B390B3093200620931F0680915106813021F080915106F4
S1234060843031F4449883E08093E40581E01BC080915106853021F080915106823031F47F
S1234080459881E08093E40582E00DC080915106833021F080915106863039F4469882E0FC
S12340A08093E40583E080935D068EEB90E0909322068093210680912606909127069F7718
S12340C00FC080912406909125068C509E4F90938B0080938A0080912606909127069068EF
S12340E09093270680932606F3C0809184009091850090930B0580930A0510928500109221
S123410084008091970590919805880F991F9093980580939705479A80918F0590919005B2
S12341208051974208F0CAC0809153069091540685369105B4F11092E4058091530690915E
S1234140540690938B0080938A0080918A0090918B009093200680931F06809151068130D5
S123416021F080915106843011F481E013C080915106853021F080915106823011F482E026
S123418009C080915106833021F080915106863029F483E080935D061092E40584E090E0B3
S12341A088C080915306909154068B5B9F4FF4F11092E40584E690E090938B0080938A0065
S12341C09093200680931F0680915106813021F080915106843029F481E080935D06459843
S12341E019C080915106853021F080915106823029F482E080935D0646980CC08091510693
S1234200833021F080915106863031F483E080935D0644981092E40588E290E0909322062E
S12342208093210684E18093100552C080915B0690915C0690938B0080938A002091240686
S1234240309125068091530690915406820F931F9093200680931F0680915106813021F09B
S123426080915106843029F481E00E941E1981E019C080915106853021F080915106823045
S123428029F482E00E941E1982E00CC080915106833021F080915106863031F483E00E9420
S12342A01E1983E08093E40584E18093100584EB90E090932206809321060AC0809124066E
S12342C0909125068C509E4F90938B0080938A002B9A7894FF91EF91BF91AF919F918F91B9
S12342E07F916F915F914F913F912F910F900FBE0F901F9018951092800081EF9FEF9093A0
S123430089008093880085EF9FEF90938B0080938A0080E88093810080EC9AED9093850091
S12343208093840083E090E090930D0580930C0580910C0590910D058068809381008091D4
S12343406F00876080936F00539852983D9A3E9A459A469A449AA2E0B2E00E94F328802DE2
S12343608093F804A1E0B2E00E94F328802D8093F9048091F9048E3039F08091F9048731E2
S123438019F087E18093F9048091690084608093690080916900816080936900E99A0895C7
S12343A021EB30E0F90110821092B6001092B2001092B300A0E7B0E08C9183608C9338984A
S12343C04098399841983A9842983B984398389839983A983B98EFE6F0E080818D7F808302
S12343E08C918C7F8C9386E0F901808384E680931B060895813099F438983B9880912D01B4
S1234400843021F439983A981092120510926F0610926E06109211051092B10008958230EC
S123442049F439983A9810926D0610926C061092120515BC08951F920F920FB60F9211245B
S12344402F933F934F935F936F937F938F939F93AF93BF93EF93FF93F89480911105843079
S123446019F481E00E94FA217894FF91EF91BF91AF919F918F917F916F915F914F913F9161
S12344802F910F900FBE0F901F9018950F931F9380912A0590912B050A9714F487E003C039
S12344A08091A10586E08093B1001092B20080918F0590919005845F914018F410925A06A6
S12344C016C080918F05909190058D56974020F08EE080935A060BC080918F0590919005D6
S12344E064E670E00E948F28655060935A06E0915A06F0E0E35DFC4F808180931301809158
S1234500A105882329F02091F3018091180108C0E0919305F0E0ED51FE4F80812091180167
S1234520829FC00111249093E8058093E70580918F05909190058059914050F580910001F5
S12345409091010182FF1AC08091E7059091E80520911901820F911D9093E8058093E705B5
S123456080912606909127068460909327068093260680911A018093E90541C080912606CE
S1234580909127068B7F909327068093260637C080912606909127068B7F90932706809341
S12345A026068091E905823050F18091E90581508093E905E091E705F091E8055091190142
S12345C02091190180911A014091E90560911A01E50FF11D90E0841B910930E070E0AC015D
S12345E0429FC001439F900D529F900D11240E948F28E61BF70BF093E805E093E705809197
S1234600A105882309F0E6C08091610687FD3EC0809161068F30D4F5E0919305F0E0EC5196
S1234620FE4F6081E0919305F0E0ED51FE4F40810091E7051091E80580914D06209161069C
S1234640E091180170E0641B710990E04AE0240290011124821B930B9C01629FC001639F61
S1234660900D729F900D11246AE070E00E94A328F0E06E9FC0016F9F900D7E9F900D112477
S1234680800F911F9093E8058093E70580914F0687FD3EC080914F068930D4F5E0919305EF
S12346A0F0E0ED50FE4F6081E0919305F0E0ED51FE4F40810091E7051091E80580915E0616
S12346C020914F06E091180170E0641B710990E04AE0240290011124821B930BAC01649F8C
S12346E0C001659F900D749F900D11246AE070E00E94A328F0E06E9FC0016F9F900D7E9F02
S1234700900D1124800F911F9093E8058093E705809100019091010184FF5CC02091560595
S123472030915705809136059091370528173907FCF48091360590913705209156053091CA
S12347405705821B930B64E070E00E94A32880919405861710F460939405809194058A3082
S123476018F089E080939405809126018093EA053091EA053430C8F08091E7059091E80507
S1234780E0919405F0E0ED5DFC4F2081820F911D9093E8058093E70531503093EA05809173
S12347A0260690912706806109C0109294051092EA0580912606909127068F7E909327061D
S12347C08093260680913605909137059093570580935605809100019091010191FD09C074
S12347E08091280586FF94C08091A105882309F48FC080911D068F5F80931D0690911D0654
S123480080911E06981708F486C010921D068091320590913305E0914F06FF27E7FDF095B3
S1234820E550FA4F208130E02817390734F480911B0690911C06890F19C08091320590914F
S12348403305E0914F06FF27E7FDF095E550FA4F208130E0821793075CF480911B061816B5
S12348603CF480911B0690911C06891B80931B0680912606909127069D7F909327068093AD
S1234880260620911B06E0914F06FF27E7FDF095E550FA4F8089332727FD309590E08C59A2
S12348A09F4F8217930754F4E0914F06FF27E7FDF095E550FA4F80898C591EC020911B061A
S12348C0E0914F06FF27E7FDF095E550FA4F4089332727FD309584E690E0841B91092817A3
S12348E03907CCF4E0914F06FF27E7FDF095E550FA4F908984E6891B80931B068091260649
S1234900909127069260909327068093260603C084E680931B068091E7059091E8052091A7
S12349204C0630E062E070E00E94A328269FC001279F900D369F900D112464E670E00E9446
S12349408F28660F771F7093E8056093E705209140053091410580911C0190E0C296281790
S123496039070CF046C0809100019091010181FF40C08091400590914105C397D4F0409190
S12349801B0180911B01209140053091410560911C0190E070E06E5C7F4FFC01E29FC00128
S12349A0E39F900DF29F900D11240E948F28461B03C080911B01482F50E08091E705909102
S12349C0E805480F591F5093E8054093E70580912101909122019093200180931F01809189
S12349E02606909127068260909327068093260611C080912606909127068D7F9093270610
S1234A008093260680911D0190911E019093200180931F018091F6059091F70583FF1CC0E6
S1234A20E091E705F091E80520913B018091E7059091E80564E170E00E94A32830E0629F9C
S1234A40C001639F900D729F900D11248E0F9F1F9093E8058093E705809100019091010170
S1234A6090FF4CC080912A0590912B05823891050CF044C08091E7059091E80520912801D1
S1234A80820F911D9093E8058093E705E0912A05F0912B05609118012091280182E890E0B5
S1234AA08E1B9F0B70E0AB01849FB001859F700D949F700D11248FEF90E0FB01E89FB00127
S1234AC0E99F700DF89F700D1124882777FD8095982F30E040E050E00E94642820E43FE1D3
S1234AE040E050E00E94B6288091E7059091E805820F931F9093E8058093E7052091E705E8
S1234B003091E8058091180145EF849FC00111248217930754F480911801849FC0011124AE
S1234B209093E8058093E7050BC08091E7059091E8051816190624F01092E8051092E7050E
S1234B408091E7059091E8059093960580939505809126069091270692FF04C0389839985A
S1234B603A983B9878941F910F9108951F920F920FB60F9211242F933F934F935F936F933C
S1234B807F938F939F93AF93BF93EF93FF93F89420911105223039F0243009F44FC0213084
S1234BA009F051C01CC080916E0690916F068F3F9105D1F1C8F180916E0690916F068F5F08
S1234BC08093B30080916E0690916F068F5F904090936F0680936E062093110534C00E94B4
S1234BE04622809195059091960590936F0680936E0680916E0690916F068F3F9105A1F0B3
S1234C0098F080916E0690916F068F5F8093B30080916E0690916F068F5F904090936F06C8
S1234C2080936E0682E007C080916E0690916F068093B30084E08093110505C081E00E948A
S1234C40FA21109211057894FF91EF91BF91AF919F918F917F916F915F914F913F912F9111
S1234C600F900FBE0F901F9018951F920F920FB60F9211242F933F934F935F936F937F9360
S1234C808F939F93AF93BF93EF93FF93F89420911205223039F0243009F453C0213009F097
S1234CA053C020C080916C0690916D068F3F910591F088F080916C0690916D068F5F87BD40
S1234CC080916C0690916D068F5F904090936D0680936C0633C080916C0690916D0687BD92
S1234CE084E024C0809195059091960590936D0680936C0624E025BD16BC80916C0690918A
S1234D006D068F3F9105A9F0A0F080916C0690916D068F5F87BD80916C0690916D068F5F41
S1234D20904090936D0680936C0682E0809312050BC080916C0690916D0687BD2093120508
S1234D4003C082E00E94FA217894FF91EF91BF91AF919F918F917F916F915F914F913F91C1
S1234D602F910F900FBE0F901F9018951F920F920FB60F9211242F933F934F935F936F93B1
S1234D807F938F939F93AF93BF93EF93FF93F89480911205843019F482E00E94FA21789461
S1234DA0FF91EF91BF91AF919F918F917F916F915F914F913F912F910F900FBE0F901F90D5
S1234DC0189554985C9855985D985498559815BCEEE6F0E080818360808384E085BD16BCB3
S1234DE082E187BD089511B88FEF84B915B887B98AB90895089508950895089588E9809302
S1234E00C10083E18093C40087EB96E09093750680937406909371068093700687E796E078
S1234E2090937306809372069093F8068093F706109276061092230608951F920F920FB679
S1234E400F9211248F939F93EF93FF9380917606882311F1E0917406F091750681918093CA
S1234E60C600F0937506E0937406E75FF64030F087EB96E090937506809374068091760641
S1234E8081508093760680917606882329F48091C1008F7D8093C100FF91EF919F918F9147
S1234EA00F900FBE0F901F9018951F920F920FB60F9211242F938F939F93EF93FF9380915F
S1234EC0C600E091F706F091F8068083809123068F5F809323068091F7069091F8060196F0
S1234EE09093F8068093F706875B964030F087E796E09093F8068093F706FF91EF919F9150
S1234F008F912F910F900FBE0F901F90189580912306882319F48FEF9FEF0895F89480910E
S1234F202306815080932306E0917206F09173062191F0937306E0937206E75BF64030F023
S1234F4087E796E090937306809372067894822F90E00895982F809176068F33E0F780917A
S1234F607606803418F080E090E00895F894809176068F5F80937606E0917006F091710613
S1234F809083809170069091710601969093710680937006875F964030F087EB96E090933A
S1234FA07106809370068091C10080628093C100789481E090E00895CF93DF93EC0104C066
S1234FC00E94AA278111219688818823C9F781E090E0DF91CF91089583E195E00E94DC27E1
S1234FE008958BE195E00E94DC2708958091230690E00895CF92DF92EF92FF920F931F936E
S1235000CF93DF93CDB7DEB729970FB6F894DEBF0FBECDBF8C01F62EE42EDE011196EEE180
S1235020F5E089E001900D928150E1F749E06E010894C11CD11CFF2081F089E090E0841B4F
S123504091092F2D30E08217930738F04150F601E40FF11D8CE28083FF244150F601E40F53
S1235060F11DC8016AE070E00E948F28805D8083C8016AE070E00E948F288B01672B11F4A3
S1235080FF2019F085E08F15B0F619E01E197E010894E11CF11C07C0F701E10FF11D808122
S12350A00E94AA271F5F1930B8F329960FB6F894DEBF0FBECDBFDF91CF911F910F91FF9052
S12350C0EF90DF90CF900895629FD001739FF001829FE00DF11D649FE00DF11D929FF00DC5
S12350E0839FF00D749FF00D659FF00D9927729FB00DE11DF91F639FB00DE11DF91FBD0145
S1235100CF0111240895991B79E004C0991F961708F0961B881F7A95C9F780950895AA1B1D
S1235120BB1B51E107C0AA1FBB1FA617B70710F0A61BB70B881F991F5A95A9F780959095D3
S1235140BC01CD01089597FB092E07260AD077FD04D0E5DF06D000201AF4709561957F4F7A
S12351600895F6F7909581959F4F0895A1E21A2EAA1BBB1BFD010DC0AA1FBB1FEE1FFF1FDC
S1235180A217B307E407F50720F0A21BB30BE40BF50B661F771F881F991F1A9469F76095BA
S12351A07095809590959B01AC01BD01CF01089597FB092E05260ED057FD04D0D7DF0AD0AE
S12351C0001C38F450954095309521953F4F4F4F5F4F0895F6F790958095709561957F4FE7
S12351E08F4F9F4F0895F999FECFB2BDA1BDF89A119600B40895F7DFE02DF5DFF02D08951B
S1235200F999FECFB2BDA1BD00BC11960FB6F894FA9AF99A0FBE0895F3DF012CF1DF112415
S12352200895FFCF2F00010002000300040005000600070008003228E803900106141E1E80
S12352403C581B581B88136419121E01010203040A0411C4098813C4096400DCE640030216
S12352600A14324696500054819596B7AFC3C8BEBEB9B0AFAFADAC4984C0CBD2D6D7D0C7B3
S1235280C2BBB8B3AEAAA9458AA2A9AAB7C0BABEBBB6B8B2B3B4B93281868DA4A58B8C8FBE
S12352A09EA6A2A6A5A6C034525D5B596F788285858281FF859FB034444E4B4A54615769A3
S12352C0727272737D9095272C1B252B334B5155616A6D6C7D828B1D211A242A32454C4F97
S12352E05E6169717E818634323232323232323232327F323232323232323232323232325B
S123530032323232323232131718191B1C1D1F21232527282C2E311418191A1C2124272B08
S12353203035393C3E414316191D232A31353B3F42484E565A5E651B1D363E525863666C7E
S12353406E777D84898D932226434B6172818A9097A8ACAFB1B6B9292E484E6B7C939BA218
S1235360AFB9BFCBD2D2D229344B536E7F9CA8B1BCC5D0D2D2D2D2283F4E587187A4B2BA36
S1235380C2D2D2D2D2D2D23746545E7691B1BEC4D2D2D2D2D2D2D239485660869FBAD2D27A
S12353A0D2D2D2D2D2D2D2000000000000000000000000000000000000000000000000002B
S12353C00000000000000000000000000000000000000000000000000000000000000000C9
S12353E0000000000000000102030405060708090A0B0C0D0E0F10010203040506070809F4
S12354000A0B0C0D0E0F100102030405060708090A0B0C0D0E0F1014161718191A1B1C1DC5
S12354201E1F2021222324191A1B1C1D1E1F2021222324252627271E1F2022232425262742
S123544028292A2B2C2D2E000204060708090A0C0E28262422201E1E1E1E1E1E1E1E1E1EF3
S12354601EF0FF80BBE0880465484BA438022BF0207019CC13860F440CC209D0074C061B07
S1235480052A046A03D1025602F201A1015F012801FB00D600B7009D00870075006600593F
S12354A0004D0044003C0034002E0029002500F0FF80BBE0880465484BA438022BF0207054
S12354C019CC13860F440CC209D0074C061B052A046A03D1025602F201A1015F012801FBF8
S12354E000D600B7009D0087007500660059004D0044003C0034002E0029002500F0FF80D7
S1235500BBE0880465484BA438022BF0207019CC13860F440CC209D0074C061B052A046A56
S123552003D1025602F201A1015F012801FB00D600B7009D0087007500660059004D0044AA
S1235540003C0034002E0029002500F0FF80BBE0880465484BA438022BF0207019CC1386C6
S12355600F440CC209D0074C061B052A046A03D1025602F201A1015F012801FB00D600B748
S1235580009D0087007500660059004D0044003C0034002E00290025000000F5047E05AE08
S12355A0066C08C00AB30D630F8B10D7118813000000000A000F001E003C007800FA0072FC
S12355C001E00180028002000008000A000C000E00C80A4A067E048403AC0D641A00200033
S12355E0270032003E0066008E00B202EB02240337034B03560361037003E800D600C2001C
S1235600B0009D008A00780078006500520040002D001900070000000100010001175A5AAD
S12356205A505050505050505050505050506400030000FA3204041B5B481B5B324A000DA4
S10F56400A002020202020202020200030
S50302B347
